:1000000000308A00D1280000831A0A28A500030EB8
:10001000A6000F288312A500030EA600A6140A0846
:10002000AD008A018313A50E0408A7002008A800CC
:100030002108A9002208AA002308AB002408AC006C
:1000400083128C308400001C27280C187528270880
:1000500084002808A0002908A1002A08A2002B0873
:10006000A3002C08A4002D088A00260E830083120A
:10007000250EA61883160900A101A201A001A30163
:100080003A08031D46283908031960281030BB00C0
:100090000310B70DB80DA00DA30D3A082302031DE0
:1000A000532839082002031C5C283908A002031CCD
:1000B000A3033A08A3020314A10DA20DBB0B482809
:1000C00000008628373084000008031974280230A5
:1000D000A100A001A00B6A28A10B69289730A000FD
:1000E000A00B7028800B672800349E308F00593099
:1000F0008E0031080319B203B1033208B800310889
:10010000B7000230BA005830B9003C282008B700C8
:100110002308B800B708031D9F28B808031D9F28AF
:10012000B6013608013C031C9F288516FA30B7003B
:1001300062208512FA30B7006220B60A9128B10811
:10014000031DBA28B208031DBA28B6013608013CBF
:10015000031CB62885160515FA30B70062208512F3
:100160000511FA30B7006220B60AA6280730B2009F
:100170000830B1000C108A1127280C30A1001F088C
:10018000C33921049F000D30A000A00BC5289F1487
:100190009F18C82883161E088312AF001E08B000DF
:1001A0001F2984011F3083051F1383161F149F14FA
:1001B0001F159F15073083129F00703083168F0024
:1001C0001830650083121F1383161F109F101F1114
:1001D0009F151F129F161F1383129F171F14B530F0
:1001E00090009E308F0059308E0083160C14C03062
:1001F00083128B04851205110730B2000830B1005C
:10020000B3013308023C031C1D2985160515AE01F8
:100210008B1BAE178B13FA30B7006220AE1B8B1707
:1002200085120511AE018B1BAE178B13FA30B70088
:100230006220AE1B8B17B30A01298512BD28300836
:10024000033C031C4429031D29292F083D3C031CA2
:100250004429051585160230B400AE018B1BAE177C
:100260008B13FA30B7006220AE1B8B17B40B2D290D
:1002700085120511AE018B1BAE178B13FA30B70038
:100280006220AE1B8B17B4293008033C031C69297C
:10029000031D4E292F08663C031C69290515851688
:1002A000AE018B1BAE178B13FA30B7006220AE1B6A
:1002B0008B17851205110230B400AE018B1BAE17EF
:1002C0008B13FA30B7006220AE1B8B17B40B5D297D
:1002D000B4293008033C031C8E29031D73292F0801
:1002E000823C031C8E2905158516AE018B1BAE17AB
:1002F0008B13FA30B7006220AE1B8B1785120511E5
:100300000430B400AE018B1BAE178B13FA30B7006C
:100310006220AE1B8B17B40B8229B4293008033C32
:10032000031CB229031D98292F089E3C031CB229E7
:100330008516AE018B1BAE178B13FA30B700622007
:10034000AE1B8B17851205110230B400AE018B1B5A
:10035000AE178B13FA30B7006220AE1B8B17B40BAD
:0C036000A629B429051185121E2963008E
:02400E00C43FAD
:00000001FF
